:030000000219FDE5
:03000B000200AA46
:03002B000201804F
:03005B0002033A63
:030073000203275E
:1000800002030406080C10182030406080040608A3
:100090000C10182030406080A0C00003070F1F0D17
:1000A0000D04050D050305030302C2AF306308C24A
:1000B0006385798AD2AF32C0D0C0E0206221E525C5
:1000C0006016E473E525F4C3334009758A00D263F2
:1000D000F57901D6F58AD262D0E0D0D0D2AF32C362
:1000E000E526334009758A00D263F57901F0F58A77
:1000F000C262E526F4603130682720720CE57BF49B
:100100005290D0E0D0D0D2AF32E57BF45290206F45
:100110001020650DE57BF4D33333335290E57B42F9
:1001200090D0E0D0D0D2AF32758A00D2637579001A
:10013000C28DD262212101C4306807206504D295A6
:10014000D29201C4306807206504D294D29101C4D0
:10015000306807206504D293D29001C4306807202C
:100160006504D295D29201C4306807206504D29408
:10017000D29101C4306807206504D293D29001C4A3
:10018000C2AFC2AD53E6EFC0D0C0E0D2D3D2AFE52C
:100190007A6009E577600575770041D4757701C20B
:1001A000CEE52A600720744F152A21F778007900E0
:1001B00020742EE580307E01F430E70278FF53DAB8
:1001C000CF207E0343DA20307E0343DA10C2D8C248
:1001D00071E580307E01F430E70279FFC3E8997061
:1001E000CB306103752A18207403752A18885CD2F5
:1001F00070E86003755F0020740DE52B6004152B1B
:10020000410743DA01C2D82070024176A85C206120
:1002100002C2702074367982B70431C3E894F0408A
:100220000374F0F8E8C4540F28F87984B703024146
:100230004CC313C3138721200802C313200A06C32B
:10024000C898F8414C28F8500374FFF88822E52D2F
:1002500054066022206B1FE536C333C333F8E564D0
:10026000C313C313F9C3952240028922E82522F55E
:100270002250037522FF7882B60459852224A824CF
:10028000C3E52495614002A861C3E895634002A8D4
:10029000638825E566700241C7C3E8AA669A5003E1
:1002A000E8FAE4F9EAC333FBE568F45B29400D257D
:1002B00067F8E56760021567400B41C70AC3E56749
:1002C0009A5002056778FF8826C26FC3E52694F826
:1002D0004002D26F20CF0AD0E0D0D043E610D2AD9A
:1002E00032C2CF053AE57A6009E578600575780095
:1002F000611D7578017801E52A6005307402152AC0
:10030000C3E55C94014005755F00611D7560007573
:100310006900E55F2401F55F5003755FFFD0E0D011
:10032000D043E610D2AD32C2AF53E67F7592FA7574
:1003300093FFC260759104D2AF32C2AF53E6EFC2F1
:10034000ADC0D0C0E0C0F0D2D3D2AFA8FBA9FCE5CD
:100350007A6007C3E913F9E813F8C2D83071026173
:10036000AC53DACF207E0343DA10307E0343DA2029
:10037000D271E580307E01F420E70261838827890D
:1003800028A1D953DACF207E0343DA20307E0343FD
:10039000DA10C2D8C271307402A1C57800E580308D
:1003A0007E01F430E702A1C5885CA1AD53DACF200D
:1003B0007E0343DA20307E0343DA10C271206102EB
:1003C000818553DACF207E0343DA10307E0343DA8F
:1003D00020C2D8D27188578958C3E89555F8E99555
:1003E00056F97B007E087A00C3E8948CE9940050AB
:1003F00005755B008177882178A2E6A8216055C346
:10040000E894C8E994005008E4D2E4FB7A0A8152E7
:10041000C3E89468E994015008E4D2E3FB7A0F81C1
:1004200052C3E894D0E994025008E4D2E2FB7A1E69
:100430008152C3E894A0E994055008E4D2E1FB7A24
:100440003C8152C3E89498E994085008E4D2E0FB58
:100450007A787E00C3E89559FCE9955AFD30E70AA1
:10046000ECF42401FCEDF43400FD755B00C3EC9A60
:0E047000ED9E5003755B018859895A855755DA
:10047E008558567802A1ADC3E89527F8E99528F975
:10048E00307C02A191307B02A191307A02A18A20A8
:10049E00750281A8E9FDE8FC81C7E9C313F9E813E9
:1004AE00F8307902A18AE9C313F9E813F83078021B
:1004BE00A18AE9C313FDE813FC20612CC3EC941C44
:1004CE00ED9402400281DEED701EC3EC94C850180C
:1004DE000529E52970021529C3E529940A5002A1C0
:1004EE00C5755C00D270A1C5E52960021529788812
:1004FE00E6F97400207F087896B90302789EE62408
:10050E00FAFEE43400FFC3EC9EFCED9FFD9208B9A9
:10051E000310A2085007207609D276A13030760259
:10052E00C276A2085016B9030DECF42401FCEDF4CA
:10053E003400FD02054A78007900A191B90315EC4B
:10054E0033FCED33FDC3EC940AFCED9400FD500436
:10055E007C007D00C3EC94FFED9400400678FF799B
:10056E0000A191EC8572F0A4C5F0A2F733F87900E2
:10057E0040030205AD78FF79000205ADE9C313F91A
:10058E00E813F8307C0EE9600278FFC3E81338F800
:10059E00E43400F9C3E894FFE99400400278FF8840
:1005AE005CD270206102A1C5741FF4552F4BF52F3C
:1005BE00C274EB7002D274752A18307403752A0A4D
:1005CE00306102A1D920740353DAFE207403752B17
:1005DE0006D0F0D0E0D0D0D2AD43E6103279010291
:1005EE0006097903020609790A020609791E02062E
:1005FE0009796402060979C80206097817E4D5E07C
:10060E00FDD8FAD9F6227A147B780206307A107B5E
:10061E008C0206307A0D7BB40206307A0B7BC80250
:10062E000630E573D5E001227902E4C291D5E0FDF2
:10063E00D294D291D5E0FDC291D5E0FDC294D29173
:10064E00D5E0FDE920E004D295D29230E004D293B9
:10065E00D290E573D5E0FDE920E002C29230E002CF
:10066E00C2907496D5E0FDD9C1EAF8D5E0FDD8FB6D
:10067E00DBB0C29122C37C007D0075F00005F0EA6C
:10068E0033FAEB33FB50F6EB13FBEA13FAC3E9FF35
:10069E00E8FEE89AF8E99BF95004EFF9EEF8B3ECAE
:1006AE0033FCED33FDD5F0DFEDF9ECF822E889F0FF
:1006BE008A20D2D4F8A9F07B0030F70B7BFFF4240C
:1006CE0001F8E9F43400F9E88520F0A4ADF0F8E97A
:1006DE008520F0A4AFF0FEED2EF974003FFA7C04F5
:1006EE00C3EA13FAE913F9E813F8DCF48BF030F7E8
:1006FE000AE8F42401F8E9F43400F9E889F0C2D4E8
:10070E00F8A9F0227882B6040302076DC3E55C9463
:10071E00014003020737852224E4F544F545F546EA
:10072E00F547F548C26E02076D7882E6FCD26EE59B
:10073E0022F523783879C7AA40AB41C3EB13FBEA05
:10074E0013FAEC146013C3EB13FBEA13FAEC141454
:10075E006007C3EB13FBEA13FAD183884489452261
:10076E00C3E5449523F8E5459400F9500CC3E8948D
:10077E0080E994FF401602079EC3E8947FE9940037
:10078E00500302079E787F790002079E788079FFDA
:10079E008849894A22E5492546F8E54A3547F985CB
:1007AE004A20E4300701F43548FA30E709C3EA94E9
:1007BE00F040150207DCC3EA940F50030207DC7801
:1007CE00FF79FF7A0F0207DC780079007AF0C3E533
:1007DE00249561500AC374019524500B0207FAE563
:1007EE004A20E70E0207FAE54A30E70688468947AF
:1007FE008A482278A5E6FAC3E54933F8E54A33F983
:10080E001206BBE930E70BC3E89480E994FF40136E
:10081E000135C3E8947FE9940050020135787F7961
:10082E00000135788079FFE820E715C3E52398F8B5
:10083E004009C3E89401400302085C780102085C99
:10084E00E8F424012523F8400302085C78FF884B66
:10085E002278A6E6FAA847A9481206BBE930E70CAB
:0E086E00C3E89401E994FF4016020891C3E824
:10087C0094FFE99400500302089178FF7900020874
:10088C0091780179FFE920E715C3E54B98F8400909
:10089C00C3E8940140030208B878010208B8E8F4F0
:1008AC002401254BF840030208B878FF88242278ED
:1008BC00FF20692879A1E76023E541601F74FF855B
:1008CC0041F0848539F0306A0375F005A4F8C5F061
:1008DC00600278FFC3E895645002A864886322C361
:1008EC00E54094C8E5419400E56350031401FC0411
:1008FC006002F563220209042275E890227883E6EF
:10090C00FF30EDF9A8BDA9BE0570C3E57094084091
:10091C0052757000E9FA79A0E76044EA7007E57156
:10092C00601B02093DC3E895716010E571500660CB
:10093C000C140209490460F9020949E571F571C307
:10094C009472401B7561C0C394044013756180C3DD
:10095C009404400B756140C39404400375610075A9
:10096C00BB0E22E5612410500274FFF5617982B749
:10097C0004022196C3A861E524985002A824C3E878
:10098C0095634002A86388258826E570B407037533
:10099C00BB1022743279A787F0A4C5F0A2F733F804
:1009AC00C3E895614002A86188228824882588269E
:1009BC008864227540007541F022C2AF75C820A82A
:1009CC00CCA9CDAA3A30CF010A75C824D2AFC3EA5C
:1009DC0013FAE913F9E813F8AB3BAC3C883B893CC0
:1009EC00C3E89BF8E99C20690A547FF93066024100
:1009FC00E5413FAD3D8A3DF9EA9D547FFA600678AA
:100A0C00FF79FF4124AE3EAF3F8B3E8C3FA83BA904
:100A1C003CC3E89EF8E99FF9C3E54113FBE540139D
:100A2C00FAE82AF540E93BF54150067540FF75415F
:100A3C00FF418CAA40AB41AC40AD417E047F02C368
:100A4C00EB9404400D1E1FC3EB94084005206A0272
:100A5C001E1FC3ED13FDEC13FCDEF7C3EA9CFAEB8F
:100A6C009DFBEF6009C3E913F9E813F8DFF7EA28F7
:100A7C00FAEB39FB8A408B4150067BFF8B408B4154
:100A8C00C3EB94025002D2663069047F0341B778FD
:100A9C0092E6FFC3E537948240110FC3E53794A06B
:100AAC0040010FC3EF940640027F057E02E541C46E
:100ABC00540FF9E541C454F0F8E540C4540F28F83C
:100ACC00C3E89EFAE99400FB4009C3EA9402EB9454
:100ADC000050047A02E4FB6131AA40AB41EBC4FE46
:100AEC00EAC4540F4EFCC3EA9CFAEB9400FBC3E837
:100AFC0013C313F8EA28FAEB3400FB8A408B41C38A
:100B0C00EB94024002C2667802EBC4FE7B00EAC49E
:100B1C00540F4EFAC3EA98FA4005C3940250027A75
:100B2C00027892E6FF3060026131855192855293D2
:100B3C00D26043E680C3E49AF8E49BF9C3E833F847
:100B4C00E933F930660261C4E8FAE9FBD3E913FD35
:100B5C00E813FC88518952C3EF94036038EF20E00E
:100B6C000DE82CF8E93DF9ECFAEDFB020B8DE828C9
:100B7C00F8E939F9C3E82402F8E93400F97AFE7B84
:100B8C00FFC3EF9403400E8A538B54884D894E8CCF
:100B9C004F8D5061F8885389548A4D8B4E8C4F8DF4
:100BAC00503069127553F07554FF754FF07550FF46
:100BBC007551F07552FF61F8E8FAD3E813FC8851CF
:100BCC00C3EF94036020EF20E007E82CF8ECFA6107
:100BDC00E4E8282402F87AFEC3EF940340088A5311
:100BEC00884D8C4F61F888538A4D8C4FE568C33320
:100BFC005002646BF5683060028102753402D26079
:100C0C0043E680E52D5406602DA840A941C3E913A5
:100C1C00F9E813F8306904E92440F9C2AF53E67FD0
:100C2C00759100C3E498F594E499F595759104D207
:100C3C006043E680D2AF22D2647543007520003049
:100C4C006C03752040020C62D26475430075204021
:100C5C00306C0375200078017901206620E52D5455
:0F0C6C00066002C2647914E541C313700104F8F5
:100C7B00C3941440027814306904781B791BC3E8C1
:100C8B0033F8C3E933F9206010E543600C30690396
:100C9B00D53404D26DA118910A0543E59B5440B598
:100CAB002002A10230690908C3E89940011881911B
:100CBB0020640A08C3E899400281628191C264C230
:100CCB00AF53E67F7591003066127594007595F001
:100CDB00759104D26043E680D2AF8162E5417EFF1D
:100CEB00C3334009C3334005C3334001FEC3E49E05
:100CFB00759400F59581DBC3E53394015002816255
:100D0B003064028162D802A1168191C26DC2AF53C9
:100D1B00E67F759100855394855495759104854DA7
:100D2B0092854E93D26043E680D2AFE52D54066098
:100D3B0008206A020533020D54306D0D206C0A2019
:100D4B0064071581158102166822780030640278D9
:100D5B0001E53775F007A4F9E5F028F5F0E9A2F005
:100D6B0013A2F113A2F213F537C39478500375371E
:100D7B0078C3E53795384007D265E57BF452903060
:100D8B006002A18A854F92855093D26043E6802200
:100D9B00207D1AC2AF754202C291C295D2923062C7
:100DAB0004D293D290D2AF759F11020FD9C2AF75F7
:100DBB004202C291C293D290306204D295D292D2A7
:100DCB00AF759F11020FD930724B207D24C2AF75C6
:100DDB004203900168757B02C290C290306206D2CA
:100DEB0094D291A1F4C294D291D2AF759F01020F0C
:100DFB00D9C2AF754203900168757B02C292C29251
:100E0B00306206D294D291C118C294D291D2AF75EE
:100E1B009F21020FD9207D1CC2AF75420390014464
:100E2B00757B02C290306204D294D291D2AF759F7F
:100E3B0001020FD9C2AF754203900144757B02C208
:100E4B0092306204D294D291D2AF759F21020FD906
:100E5B00207D1AC2AF754204C292C293D290306207
:100E6B0004D294D291D2AF759F21020FD9C2AF7524
:100E7B004204C290C295D292306204D294D291D2E3
:100E8B00AF759F01020FD930724B207D24C2AF7515
:100E9B00420590015C757B04C291C291306206D20F
:100EAB0095D292C1B4C295D292D2AF759F11020F57
:100EBB00D9C2AF754205900174757B01C291C29185
:100ECB00306206D293D290C1D8C293D290D2AF7572
:100EDB009F11020FD9207D1CC2AF754205900138BE
:100EEB00757B04C291306204D295D292D2AF759FBA
:100EFB0011020FD9C2AF754205900150757B01C22B
:100F0B00913062E8D293D290D2AF759F11020FD974
:100F1B00207D1AC2AF754206C290C294D291306244
:100F2B0004D295D292D2AF759F01020FD9C2AF7581
:100F3B004206C292C294D291306204D293D290D222
:100F4B00AF759F21020FD930724C207D24C2AF7533
:100F5B004201900174757B01C292C292306206D23B
:100F6B0093D290E174C293D290D2AF759F21020FAE
:100F7B00D9C2AF75420190015C757B04C290C290DF
:100F8B00306207D295D292020F99C295D292D2AF0C
:100F9B00759F01020FD9207D1CC2AF7542019001D4
:100FAB0050757B01C292306204D293D290D2AF754E
:100FBB009F21020FD9C2AF754201900138757B0496
:100FCB00C290306204D295D292D2AF759F01C265A6
:100FDB0022900136757B00C292C291C290C292C21E
:100FEB0091C290C26222788076090876090876044D
:100FFB000876FF0876030876FF08760A087603085A
:10100B007601087601788C76010876FF0876FF0862
:10101B0076FF0876FF0876FF0876030876FF0876DA
:10102B00FF0876FF0876250876D0087628087650D4
:10103B000876040876FF08760208760008767A08A8
:10104B0076FF0876010876010876000876030876A5
:10105B0000227887E6FFC272BF0302D2727888E65D
:0F106B00C394036008C27DE630E102D27DC27EED
:10107A007889E630E102D27EC3EF94026008758E69
:10108A0001D273021095758E00C273227880E6141D
:10109A009000809378A5F67881E614900080937882
:1010AA00A6F67886E61490008D9378A7F67886E6F9
:1010BA00F539C394025003753902789CE67538FFF6
:1010CA00B402037538A0B4030375388278A3E61412
:1010DA0090009A93F566120FDC22227896E6FA7847
:1010EA0097E6FB7888E6B40305C3EB940EFB307FE2
:1010FA00047A007BFFC3EB9AFCC3948250027C8281
:10110A007572000572EC8572F0A4C3E5F0947D4017
:10111A00F222D27F11E51205FA1205FA7A007B0053
:10112A007C101205F0E55C2AFA74003BFBDCF37CC8
:10113A0004C3EB13FBEA13FADCF7FEC27F11E522C4
:10114A00757C00757D00E5EF20E60375200005201B
:10115A00903FFFE520146006901FFF14600093047F
:10116A00600375EF1653D9BF7581C043FF8012051E
:10117A00EB75EF0643B203E5B3240220E70DF52130
:10118A00E5E320E0068521B343E301120FDC758015
:10119A00FF75A40075F19175D47F75900075A53F10
:1011AA0075F23F75D50075A60175E241120FDCE4B0
:1011BA00F8F6D8FD756801120FF11216C7789886ED
:1011CA0073753001C2AF1206041206141205FA1220
:1011DA00061B1205FA1206221205FAC2AF757C0026
:1011EA00757D0078FA79FA308707D9FBD8F7021C9F
:1011FA0000115D119611E411E578988673120FDCDF
:10120A0075A90075B680757A00758810758902759A
:10121A00C82475910475D84075A82275B80275E678
:10122A0090759B80759D0075D10E75BCC075BB0EFF
:10123A0075BA1175E8801205EBD2AF12090175363D
:10124A000053DACF207E0343DA20307E0343DA10DC
:10125A0043DA01C2D8C271120604D2617B037A0C46
:10126A00E55B70077A0CDB030211E51205FA2070C0
:10127A00030211E5C270E55CC3940240E1E52F5414
:10128A001F855E5DF55EB55DD5DAD5C26153DACFED
:10129A00207E0343DA20307E0343DA10C2D8C271BB
:1012AA0078A2E67008D274E52F54E0F52FC275755E
:1012BA0029001205FF307409C3E529940A4002D2B5
:1012CA00751205F078023074027800C3E55C984024
:1012DA00F0C2AF120614120614120614D2AF120686
:1012EA0004754C007888E6B4030261E11205F078CF
:1012FA008CE6C3940150030213E1E530C394015014
:10130A00030213E1757CA5757DF1207435C3E55C94
:10131A0094FF50030213E1C2AF120629D2AF12059D
:10132A00FFC3E55C940150EFC2AF1206141205F533
:10133A00120614D2AF1205FFC3E55C94FF40E9021E
:10134A00187F7F02D27F11E51205FFC2AFC27F115B
:10135A00E5AE5CC3E55C947FD2AF500261F1120541
:10136A00EBC2AF120629D2AFDFDA311CC3EE78978F
:10137A00F61206041218027F0AD27F11E51205FF3F
:10138A00C2AFC27F11E5AE5CC3E55C947FD2AF50B9
:10139A00E61205EBC2AF1206141205F5120614D2B4
:1013AA00AFDFD6311CEE24037896F6F87997E7C3B7
:1013BA0094824003985006E824827897F61206042D
:1013CA001217151218311205FF11E5C3E55C94FFD7
:1013DA005002610E02187F757C00757D00C3E55CC2
:1013EA00954C4003855C4C1205FF78017988E7B477
:1013FA0003027805C3E55C98400241EEC2AF1206CB
:10140A0029120629120629D2AF120604753000E401
:10141A00F531F5320531E531F4703F0532789AE657
:10142A007819146012783214600D787D1460087887
:10143A00FA146003753200C3E53298401D120FDCBE
:10144A001205EB153275310078998673C2AF120610
:10145A0029D2AF789886731205FF1205F5E52A702E
:0E146A000530740221E578012074027806C373
:10147800E55C9840A17888E6C3940360031205FFF1
:10148800E52A70030211E5C2AF120FDCE4F522F57C
:1014980023F524F525F526F567D2AF7885E6C3331D
:1014A800F565E4F544F545F546F547F548F570F575
:1014B8002CF52DF53775700875BB101205EB120960
:1014C8000530EDFDA8BDA9BEE97001F888711209C3
:1014D8000975700875BB10115DC2AF7561FF1209FF
:1014E8009F852261852262852263D2AF75220175AC
:1014F8002401752501752601856069756A0175B62F
:101508009075A903757A017888E6B40307C27D301F
:101518007602D27DD268D269753300120F1B120F82
:10152800521209BF1209C61209BF1209C61209BF11
:10153800120C54120712120D55120D9B1209C612E5
:101548000C43306E0312076E2066031208BB306628
:10155800031208EB120D55120DD21209C6120C54C3
:10156800306E031207A3120D55120E5B1209C61234
:101578000C43306E03120801120D55120E92120917
:10158800C6120C54306E0312085F120D55120F1B51
:101598001209C6120905120C43120D55120F5212E8
:1015A80009091209C63069328564618564628560FB
:1015B80069756A0179187A0CC3E53399400FC269D5
:1015C800D26A8A358564618564630215E2C3E55C85
:1015D80094014003021538021670306A25206C22E7
:1015E800E535147006C26AD26BA138F535C3E55CDF
:1015F800940140030215387888E6C3940360030217
:10160800167075360078FA79A4E760027803C3E5A6
:101618005F985054307404E52A604D7888E6B40326
:1016280017207D05207607C140307602C140206C26
:1016380007D26C856461A17778F0306C05856461A8
:101648007820C3E541985002A138306C1BC26CC2A7
:101658007D307602D27DD26A753512856461A138F3
:101668000536E55C6002C173753600C2AF120FDC47
:101678007887E6FE7602115D7887EEF6E4F522F5C6
:1016880023F524F525F526F565752C00752D0075CF
:10169800A90075B680757A00D2AF1205FF120FDC6B
:1016A80078A4E6600CC295D292C294D291C293D229
:1016B80090307409C3E5369404400221E5811990FD
:1016C8001A0D7820121757E520B4550CA312175796
:1016D800E520B4AA030216F5757CA5757DF1120FF5
:1016E800F1121715757C00757D00021714901A0306
:1016F80078807B0A121757A308DBF9901A0F788CA9
:101708007B19121757A308DBF9901A2822C2AF12C7
:10171800179A121777901A00740E12175CA374099F
:1017280012175CA3741512175C901A0378807B0A51
:1017380012175BA308DBF9901A0F788C7B19121724
:101748005BA308DBF91217AD12178B901A2822E455
:1017580093F622E6438F01538FFDFFC3E583941C64
:10176800400122EF857CB7857DB7F0538FFE224379
:101778008F02438F01857CB7857DB7901A0DF05392
:101788008FFC22901A0D7455F15C901A0E74AAF110
:101798005C227A3079D07820901A40F157E520F70A
:1017A80009A3DAF7227A3079D0901A40E7F15C0978
:1017B800A3DAF922AB74A875BB01027980BB0202D7
:1017C8007981BB03027982BB04027984BB05027963
:1017D80086BB06027992BB07027987BB080279A308
:1017E800BB0902799CBB0A027988BB0B027989E89C
:1017F800F7227C05120604DCFB22C2AF1206141283
:10180800061B1206221206291205F51206141206E4
:101818001B1206221206291205F512061412061BBF
:10182800120622120629D2AF22C2AF1206291206C8
:101838002212061B1206141205F512062912062298
:1018480012061B1206141205F51206291206221298
:10185800061B120614D2AF22AE74AF75C2AF1206C1
:0F186800141206141206141205F5DEF2120629E8
:101877001205F5DFF8D2AF2211021217FA1217FA82
:1018870075740175750175760011607C05AD5C1284
:101897000604C3ED955C70F5C3E55C9401400AC38B
:1018A700E55C94FF40360218C01217BC12171511D9
:1018B70002C2AF75EF161217FADCD20576C3E576CA
:1018C7009403500280C31217FA0575E5741490004B
:1018D7009F93F808C3E57598500280AA1217FA1269
:1018E70017FA0574C3E574940C50028096120FF131
:0B18F700121715C2AF75EF161217FA9A
:0319FD0002114A8A
:101A00000E0915090904FF03FF0A03010155AA0184
:101A1000FFFFFFFFFF03FFFFFF25D0285004FF0259
:091A2000007AFF0101000300FF40
:101A400023454D41585F4C746E675F32304123200F
:101A500023424C48454C492346333930232020202B
:101A60002020202020202020202020202020202076
:101C0000C2AFC2D353D9BF7581C043B20343FF8073
:101C1000752438752503B1DC7529A5752AF175E29F
:101C20004043F18053A47F75D4FFD2877DFA7803B7
:101C300079E67C10752200752300901DE97B0675FE
:101C400024987525013087028145208708D8FBD963
:101C5000F9DCF781B7308708D8FBD9F9DCF781B711
:101C6000B19CE493A3C39A6004DDC381B7DBDBB10D
:101C70008E6002812E7B08E493FAA3B16FDBF87AC1
:101C800030B16F752200752300B18EEAFCEBFDC305
:101C9000ED94FE400EB18E8A278B28ED30E0048A49
:101CA000828B83B18E7AC270D8C3ED94FE601950D6
:101CB000CEBD002BEC600F7520007521FF7529004B
:101CC000752A000200008100A827A9280809D80465
:101CD000D90281DCB192EA89AAF281CE0D81A3C337
:101CE000ED94035053EDA2E092007AC5C3E58294CF
:101CF00000E583941C508A200010438F02438F011B
:101D00008529B7852AB7F0300029A827A92808090E
:101D1000438F01538FFDD804D902A133C3E58394C7
:101D20001C4003A3A11689AAE28529B7852AB7F02A
:101D3000A3A116538FFC817F7AC1BD030CE493A34A
:101D4000FAB153DCF8B14B817F8181AA22AB23B178
:101D50006FEBFAEA6222752608C3E52313F523E543
:101D60002213F52250066323A0632201D526EAB18F
:101D7000DCB1DC75260AEAF4200102D287300102C8
:101D8000C287B1DCC3134002C201D526EB22B19257
:101D9000EAFB208702A192308702A197752608AE40
:101DA00024AF25C3EF13FFEE13FEB1E0B1DCC3EAAD
:101DB000133087024480FA30E703632201C3E5232E
:101DC00013F523E52213F52250066323A0632201B5
:101DD000D526D9E52265236523F52222AE24AF2539
:101DE0000E0FDEFEDFFCD20122424C48656C6934E6
:071DF000373164F390060196
:00000001FF
